:10000000502D0010E9000000ED000000EF0000009E
:10001000F1000000F3000000F500000012CDFFEF3A
:10002000000000000000000000000000F7000000D9
:10003000F900000000000000FB000000FD000000CF
:10004000FF000000B9210000FF000000FF000000D9
:10005000FF000000FF000000FF000000FF000000A4
:10006000FF000000FF000000FF000000FF00000094
:10007000FF000000FF000000FF000000FF00000084
:10008000FF000000FF000000FF000000FF00000074
:10009000FF000000FF000000FF000000FF00000064
:1000A00051250000FF000000FF000000FF000000DD
:1000B000FF000000FF000000FF000000FF00000044
:1000C000FF000000FF000000FF000000DFF80CD080
:1000D00000F05AF80048004741310000502D001050
:1000E000D0F800D0D0F804F005480047FEE7FEE75E
:1000F000FEE7FEE7FEE7FEE7FEE7FEE7FEE7FEE7D8
:10010000CD00000010B50B4604461146184600F01D
:1001100027F8C4E9000110BD40EA01039B0703D0A2
:1001200009E008C9121F08C0042AFAD203E011F836
:10013000013B00F8013B521EF9D27047D2B201E0F8
:1001400000F8012B491EFBD270470022F6E710B5DC
:1001500013460A4604461946FFF7F0FF204610BD35
:1001600070B500242546002801DA01244042002908
:1001700001DA0125494200F019F8AC4200D04042B2
:10018000002C00D0494270BD064C074D06E0E068E7
:1001900040F0010394E8070098471034AC42F6D3CE
:1001A000FFF798FF8C3B0000AC3B000030B50B46DE
:1001B000014600202022012409E021FA02F59D4297
:1001C00005D303FA02F5491B04FA02F52844151E6B
:1001D000A2F10102F1DC30BD70B5044600BF00BFE2
:1001E00000BF00BF00BF00BF00BF00BF00BF00BF17
:1001F00000BF00BF00BF00BF00BF00BF00BF00BF07
:1002000000BF00BF00BF00BF00BF00BF00BF00BFF6
:1002100000BF00BF00BF00BF00BF00BF40251C4E95
:10022000F561D72001F0CCFE002001F0C9FE20705E
:10023000B56100BF00BF00BF00BF00BF00BF00BF6F
:1002400000BF00BF00BF00BF00BF00BF00BF00BFB6
:1002500000BF00BF00BF00BF00BF00BF00BF00BFA6
:1002600000BF00BF00BF00BF00BF00BF00BF00BF96
:1002700000BF207800F03D012C2902D04FF0FF3064
:1002800070BD000601D5002070BD012070BD0000CA
:1002900000C009204FF4047070474FF404107047F9
:1002A000F8B5084E0546B46805E0B068001BA842E2
:1002B00001D30120F8BD6846FFF78EFF0028F4D176
:1002C000F8BD00000000094004490020086004490E
:1002D00008607846034908600020704780000010DD
:1002E00084000010880000100020704701460007BD
:1002F000C00E090600D5401C70477047FFFFFFFF86
:1003000070B500BF00BF00BF00BF00BF00BF00BF8F
:1003100000BF00BF00BF00BF00BF00BF00BF00BFE5
:1003200000BF00BF00BF00BF00BF00BF00BF00BFD5
:1003300000BF00BF00BF00BF00BF00BF00BF00BFC5
:1003400000BF40241E4DEC6104211E4801F042FE16
:10035000AC6100BF00BF00BF00BF00BF00BF00BF57
:1003600000BF00BF00BF00BF00BF00BF00BF00BF95
:1003700000BF00BF00BF00BF00BF00BF00BF00BF85
:1003800000BF00BF00BF00BF00BF00BF00BF00BF75
:1003900000BF0D48FFF784FF0C490D4A0D4B38B1E3
:1003A000822008602220106078461860822070BD8C
:1003B00000200860106078461860002070BD0000C2
:1003C00000C009201C3B000000B4C40480000010E1
:1003D0008400001088000010074800210167C160F8
:1003E000102242618161F122C2630448826804489C
:1003F000C0E9002108467047008000400000094025
:10040000DC0000104D0B00002DE9F04FADF5057D2F
:1004100000BF00BF00BF00BF00BF00BF00BF00BFE4
:1004200000BF00BF00BF00BF00BF00BF00BF00BFD4
:1004300000BF00BF00BF00BF00BF00BF00BF00BFC4
:1004400000BF00BF00BF00BF00BF00BF00BF00BFB4
:100450004024DFF8EC914D46C9F81C40D72001F04C
:10046000AFFD002001F0ACFDAC6100BF00BF00BFDC
:1004700000BF00BF00BF00BF00BF00BF00BF00BF84
:1004800000BF00BF00BF00BF00BF00BF00BF00BF74
:1004900000BF00BF00BF00BF00BF00BF00BF00BF64
:1004A00000BF00BF00BF00BF00BF00F03D00654DB2
:1004B000654E664F4FF0820B2C2854D100BF00BF11
:1004C00000BF00BF00BF00BF00BF00BF00BF00BF34
:1004D00000BF00BF00BF00BF00BF00BF00BF00BF24
:1004E00000BF00BF00BF00BF00BF00BF00BF00BF14
:1004F00000BF00BF00BF00BF00BF00BFA046CA468C
:10050000C9F81C409F2001F05BFD002001F058FD60
:10051000C4B2002001F054FDC0B2C9F8188000BF79
:1005200000BF00BF00BF00BF00BF00BF00BF00BFD3
:1005300000BF00BF00BF00BF00BF00BF00BF00BFC3
:1005400000BF00BF00BF00BF00BF00BF00BF00BFB3
:1005500000BF00BF00BF00BF00BF00BF00BF1F2C17
:1005600001D126280AD02120C5F800B03060784695
:10057000386082200DF5057DBDE8F08F4FF4057BD6
:10058000FF2259466846FFF7D9FD87208DF8000005
:1005900000248DF801408DF802408DF8034000BF23
:1005A00000BF00BF00BF00BF00BF00BF00BF00BF53
:1005B00000BF00BF00BF00BF00BF00BF00BF00BF43
:1005C00000BF00BF00BF00BF00BF00BF00BF00BF33
:1005D00000BF00BF00BF00BF00BF00BF00BFC146DB
:1005E0004046D046CAF81C005946684601F0F2FC65
:1005F000C8F8189000BF00BF00BF00BF00BF00BF19
:1006000000BF00BF00BF00BF00BF00BF00BF00BFF2
:1006100000BF00BF00BF00BF00BF00BF00BF00BFE2
:1006200000BF00BF00BF00BF00BF00BF00BF00BFD2
:1006300000BF00BF2C60784634603860002099E726
:1006400000C0092080000010840000108800001005
:100650002DE9FE4F454E464FDFF818815FEA02094B
:100660008A4615D001464FF4047201A8FFF74AFDEF
:10067000DDE901544048FFF713FE90B1822030605D
:100680002120794638608220C8F80010BDE8FE8F2E
:10069000862030600920794638608620C8F800102E
:1006A000F4E7E8208DF80000A8098DF80100A80003
:1006B00040EA24208DF802008DF8034000BF00BFFF
:1006C00000BF00BF00BF00BF00BF00BF00BF00BF32
:1006D00000BF00BF00BF00BF00BF00BF00BF00BF22
:1006E00000BF00BF00BF00BF00BF00BF00BF00BF12
:1006F00000BF00BF00BF00BF00BF00BF40241F4DB0
:10070000EC610421684601F065FC0421684601F0B3
:100710004BFC4946504601F047FCAC6100BF00BFAE
:1007200000BF00BF00BF00BF00BF00BF00BF00BFD1
:1007300000BF00BF00BF00BF00BF00BF00BF00BFC1
:1007400000BF00BF00BF00BF00BF00BF00BF00BFB1
:1007500000BF00BF00BF00BF00BF00BF002030606F
:1007600079463860C8F8001090E70000800000105B
:100770008400001088000010A086010000C009203D
:100780002DE9F04FADF5137D0C46DDF870820026A3
:10079000DFF80C94DFF80CA4DFF80CB415468B934B
:1007A0005FEA08012AD04FF4047701463A4685A84B
:1007B000FFF7A8FCDDE985018D918A903A46611C1E
:1007C00085A8FFF79FFCDDE9850188918C903A466A
:1007D00029468EA8FFF796FCDDE98E5401A88E907D
:1007E000F248FFF75DFDB8B182212220C9F8001060
:1007F000CAF800007846CBF8000006E18620C9F868
:10080000000009207946CAF800008620CBF80010C5
:100810000DF5137DBDE8F08FA8EB0607C4F5047055
:10082000B84200D207462CB18A9885427ED18D9875
:1008300084427BD1FF224FF405716846FFF77EFCAE
:1008400087208DF8000000208DF801008DF802004F
:100850008DF803008A9885420FD18D9884420CD17F
:1008600005EB45102246000101A9FFF7F1FE8B9828
:100870003A4681198E98204403E08B983A468119B4
:1008800001A8FFF749FC8C9885420BD1889900EBB1
:10089000401001EB0010C1F504720B468E9919440B
:1008A000FFF7D6FE00BF00BF00BF00BF00BF00BF04
:1008B00000BF00BF00BF00BF00BF00BF00BF00BF40
:1008C00000BF00BF00BF00BF00BF00BF00BF00BF30
:1008D00000BF00BF00BF00BF00BF00BF00BF00BF20
:1008E00000BF00BF4021B248C1614FF405716846A6
:1008F00001F070FBAE494020886100BF00BF00BF1F
:1009000000BF00BF00BF00BF00BF00BF00BF00BFEF
:1009100000BF00BF00BF00BF00BF00BF00BF00BFDF
:1009200000BF00BF00BF00BF00BF00E00AE000BF83
:1009300000BF00BF00BF00BF00BF00BF00BF002C52
:100940007ED0C0E055208DF80000A8098DF8010088
:10095000A8008DF8020000208DF8030000BF00BF42
:1009600000BF00BF00BF00BF00BF00BF00BF00BF8F
:1009700000BF00BF00BF00BF00BF00BF00BF00BF7F
:1009800000BF00BF00BF00BF00BF00BF00BF00BF6F
:1009900000BF00BF00BF00BF00BF00BF40218448B0
:1009A000C1610421684601F015FB8149402088613E
:1009B00000BF00BF00BF00BF00BF00BF00BF00BF3F
:1009C00000BF00BF00BF00BF00BF00BF00BF00BF2F
:1009D00000BF00BF00BF00BF00BF00BF00BF00BF1F
:1009E00000BF00BF00BF00BF00BF00BF00BF00BF0F
:1009F0006E48FFF755FC50B18221C9F80010222043
:100A00007946CAF80000CBF80010822000E7872062
:100A10008DF8000000208DF80100200A8DF80200FA
:100A20008DF8034000BF00BF00BF00BF00BF00BF84
:100A300000BF00BF00BF00BF00BF00BF00BF00E09D
:100A400047E000BF00BF00BF00BF00BF00BF00BF46
:100A500000BF00BF00BF00BF00BF00BF00BF00BF9E
:100A600000BF00BF00BF00BF40205149C861042142
:100A7000684601F0AFFA8B983946304401F0AAFA83
:100A80004B494020886100BF00BF00BF00BF00BFCE
:100A900000BF00BF00BF00BF00BF00BF00BF00BF5E
:100AA00000BF00BF00BF00BF00BF00BF00BF00BF4E
:100AB00000BF00BF00BF00BF00BF00BF00BF00BF3E
:100AC00000BF00BF00BF8A98854204D18D98844240
:100AD00001D1862000E089208DF80000A8098DF85A
:100AE0000100A8008DF8020000208DF8030000BF6F
:100AF00000BF00BF00BF00BF00BF00BF00BF00BFFE
:100B000000BF00BF00BF00BF00BF00BF00BF00BFED
:100B100000BF00BF00BF00BF00BF00BF00BF00BFDD
:100B200000BF00BF00BF00BF00BF00BF00BF402428
:100B30001F48C4610421684601F04CFA1C488461D6
:100B400000BF00BF00BF00BF00BF00BF00BF00BFAD
:100B500000BF00BF00BF00BF00BF00BF00BF00BF9D
:100B600000BF00BF00BF00BF00BF00BF00BF00BF8D
:100B700000BF00BF00BF00BF00BF00BF00BF00BF7D
:100B80003E4400246D1C4645FFF42AAE0020C9F8FF
:100B900000007946CAF80000CBF8001038E60000E3
:100BA000800000108400001088000010A086010062
:100BB00000C009200948816809480268891A42680A
:100BC00002EB4203C3EBC212B1EBC20F04D3054ADE
:100BD000022151600021416070470000000009407F
:100BE000DC0000100080004070B541F28832904275
:100BF00015D8642800D290B942F2107291420ED8F2
:100C000005290CD30F4CA2680F4B1D68521B5D6861
:100C100005EB4506C6EBC515B2EBC50F01D20020AA
:100C200070BD0A4A0225556040B1094EB6FBF0F08E
:100C300040109061D061556001205060A068C3E908
:100C40000001ECE700000940DC00001000800040DB
:100C500080A8120170B50B4C00250E466560FFF7A9
:100C6000C3FF094A06EB46012068C1EBC611936831
:100C70001B1AB3EBC10FFAD30449022048600020CD
:100C8000656070BDDC00001000000940008000407D
:100C900070B50023084D0AE0CE5C04885B1C86EA30
:100CA00014269BB235F8166086EA04240480521E8E
:100CB00092B2F1D270BD0000083600002DE9FC416F
:100CC0000746002090460E46ADF8000004460EE0B0
:100CD000351B402D00D9402539192A460D4800F012
:100CE0009CFBAAB20B496846FFF7D2FF2C44B442E2
:100CF000EED33919424601A800F08FFBBDF8000081
:100D0000BDF80410884202D10120BDE8FC8100201A
:100D1000FBE70000140100102DE9F041684C0027AA
:100D20008CB0A770E770DFF89C814FF400562771F4
:100D3000012519223146684600F06FFB0222162178
:100D40003046FFF7BBFF00287DD0DDF80E100222F1
:100D500006F11900FFF7B2FF002874D09DF80000DB
:100D600006282ED2DFE800F02E03032E2E1CD8F822
:100D70007420DDF80A30521C934222D2D8F8741045
:100D8000DDF80A30C91ADDF80E30491C994218D333
:100D9000DDF80A10DDF80E301944914211D811E047
:100DA000DDF80E10B1F5F42F00D9A570DDF81210A2
:100DB000C1F30B41502905D0DDF81210B1F1107FBD
:100DC00000D0A570012803D0022801D0052839D110
:100DD000022206F21D4109A8099700F01EFB09999D
:100DE000019889B2884200D0A570012206F22541FF
:100DF00009A8099700F011FB0999BDF80100C9B2D3
:100E0000884200D0A5709DF8000002281AD1042263
:100E100006F2494109A8099700F0FFFADDF812002F
:100E20000999884200D0A570012206F24D4109A817
:100E3000099700F0F2FA09999DF80300C9B28842B7
:100E400000D0A57000E023E09DF81800401EFE28A9
:100E500000D2A570BDF80100A0F57F41FF3901D097
:100E60003E2802D19DF8030020B9684600F0E8F959
:100E700000B9A570DDF80E001B360644684600F088
:100E8000DFF930B1E07880B1217988420DD012E0ED
:100E9000A5709DF8180010B92079401C2071E078E9
:100EA000401CC0B2E0700C2801D3A57003E0A0780C
:100EB00000283FF43EAFA0780CB0BDE8F081000000
:100EC0000C000010C039000070B500F049F810495E
:100ED000104D114E114C087050B1114900EBC0007B
:100EE00001EB800080688047000609D5206870BD4E
:100EF000822020602120286078463060822070BDEA
:100F000000202060286078463060002070BD00001E
:100F100010010010840000108800001080000010F4
:100F2000203B00000948007828B1094900EBC000C7
:100F300051F8200000470749822008600649212017
:100F4000086078460549086082207047100100104B
:100F5000203B00008000001084000010880000107A
:100F600070B5002400BF00BF00BF00BF00BF00BFBE
:100F700000BF00BF00BF00BF00BF00BF00BF00BF79
:100F800000BF00BF00BF00BF00BF00BF00BF00BF69
:100F900000BF00BF00BF00BF00BF00BF00BF00BF59
:100FA00000BF00BF40251F4EF5619F2001F008F8EB
:100FB000002001F005F860F30704002001F000F8BC
:100FC00060F30F24002000F0FBFF60F31744B561CD
:100FD00000BF00BF00BF00BF00BF00BF00BF00BF19
:100FE00000BF00BF00BF00BF00BF00BF00BF00BF09
:100FF00000BF00BF00BF00BF00BF00BF00BF00BFF9
:1010000000BF00BF00BF00BF00BF00BF00BF00BFE8
:10101000A4F21F64B4F5005F01D0002070BD012070
:1010200070BD000000C00920054982200860054904
:10103000222008607846044908608220704700003A
:1010400080000010840000108800001005498220F4
:10105000086005492120086078460449086082201C
:10106000704700008000001084000010880000100D
:101070000549822008600549222008607846044915
:10108000086082207047000080000010840000107B
:10109000880000102DE9F041144B154D154E1B78BA
:1010A000154C63B19AB1154F03EBC30307EB8303F0
:1010B0001B699847000612D52068BDE8F0818220A0
:1010C000206021202860784630608220F5E7862065
:1010D000206009202860784630608620EDE70020F7
:1010E00020602860784630600020E6E7100100109C
:1010F000840000108800001080000010203B0000D9
:10110000F8B5184C184D194E2778194CDDF818C051
:1011100087B1BCF1000F15D0CDF800C0DFF854C086
:1011200007EBC7070CEB8707FF69B847000611D527
:101130002068F8BD82202060222028607846306038
:101140008220F8BD86202060092028607846306023
:101150008620F8BD0020206028607846306000209E
:10116000F8BD00001001001084000010880000107D
:1011700080000010203B000070B50948022400F1F7
:101180001F05816829B1007B000607D4022001F009
:10119000B3FC2C7300F006FC002070BD012070BD74
:1011A000AD1B001010B50C480C4C8068A17888422B
:1011B00000D2A0700849A2784039822001F0CCFC0E
:1011C000032060700448A2781F308168891A81600A
:1011D0000021017310BD0000AD1B00108C00001039
:1011E0002DE9F041092000F04BF8124800264FF499
:1011F0007A770670C8213846FFF72CFD0E4CA068A0
:1012000042F21075A168091AA942FBD3C8213846D9
:10121000FFF720FDA068A168091AA942FBD3C821E5
:101220003846FFF717FD0548022186708171C670A8
:10123000BDE8F0817C000010000009400C000010A7
:101240000021425C12B9491C1829FAD3182901D08F
:10125000002070470120704701460020074ACB0755
:1012600003D0536DDB0600D50120890704D5516DED
:10127000890601D540F002007047000000C0092037
:1012800070B54F4B50B15968042403250226052937
:1012900007D2DFE801F0072D4C7491000020586060
:1012A000986070BD042807D0052809D001240228C1
:1012B0007DD0012809D011E0032000F085F848E036
:1012C000BDE87040012000F07FB8032000F07CF8FA
:1012D0000CE000BF00F086F85C6070BD0E28FCD109
:1012E000032000F071F8022000F07CF80120F1E703
:1012F00006280AD0032810D00A2813D0092811D0B4
:101300000D280FD00C28D7D070BD032000F05CF85A
:10131000022000F067F85E6070BD032000F054F812
:10132000012028E0032000F04FF8022012E00628F8
:1013300014D00A281BD00928C7D00C28BCD00D28EF
:10134000F0D00F28E8D1032000F03EF8022000F092
:1013500049F80120BDE8704000F044B8986810F0EA
:101360001F0F00F101009860D6D102201BE003207E
:1013700000F02AF8022000F035F85D6070BD072803
:1013800006D00A2898D00B2811D009289DD070BD0E
:10139000022000F019F8986810F03F0F00F10100EA
:1013A0009860F4D10120BDE8704000F029B8032016
:1013B00000F00AF802208DE70628A6D08EE700008C
:1013C000CC000010002070470549C20701D0102250
:1013D000CA65800701D52020C8650020704700003D
:1013E00000C009200549C20701D010228A65800784
:1013F00001D52020886500207047000000C009202A
:1014000010B50446FFF728FF0346FFF7DDFF24EA87
:101410000300FFF7E7FF002010BD10B50B460146A3
:1014200000241846FFF736FE204610BD0E4810B5C2
:101430004178022908D003290ED0042910D00529AB
:1014400001D10021417010BD0848C07B2828FAD185
:10145000BDE8104000F034B9BDE8104000F0A2BA79
:10146000822001F049FBF7E78C000010AD1B001053
:1014700010B51449022001F049F9134988704878E1
:1014800060B101280ED0022001F036FB0D49022088
:101490005F310873BDE8104000F084BABDE8104029
:1014A00000F014B807484030C07B2A2805D02F2808
:1014B00007D1BDE8104000F035B9BDE8104000F09C
:1014C00075B910BD6D1B00108C0000102DE9F041A6
:1014D0004A4D4B4C0021A878A4F1400202E0535C35
:1014E0006354491C03468142F9D31F2B7CD12068E9
:1014F0004449884278D1424E60681F364FF0010857
:101500007060A068B060607B18B9A07B08B110283B
:1015100002D986F80C8063E0E07B1E28F9D011DC4C
:10152000122833D006DC68B30328F2D1BDE8F041BD
:1015300000F00EBA1528ECD01A28EAD1BDE8F04127
:1015400000F07EB902272A282ED011DC232821D0D2
:10155000252823D02828DCD100F08AF900282CD0B7
:10156000207B00061ED56F70BDE8F04100F0A8B8E2
:101570002F2824D05528CCD05A28CAD1BDE8F04114
:1015800000F042B9BDE8F04100F01EBABDE8F041FC
:1015900000F03AB8BDE8F04100F0B4B9BDE8F04160
:1015A00000F08EB9022018E000F062F9002804D0A3
:1015B000207B000610D485F80180BDE8F08100F0A2
:1015C00057F90028F9D0207B000605D485F8018062
:1015D000C5F82880F1E707E0822001F08DFA377323
:1015E000BDE8F04100F0DEB9822001F085FA02206A
:1015F00001F082FA06206870DFE700008C0000101E
:10160000AD1B0010555342431CB5FFF7B5FD002834
:101610004ED028480A2206210388684601F0F2FECF
:101620002548002280230270437082700121C1701E
:101630002021017143718271C271412202725422D0
:1016400042724F2282724C22C272017341738173C3
:10165000C173462202745023437472238374692336
:10166000C3746E230375742343758175C2756C2230
:10167000027661224276732282766822C2760177F0
:1016800041778177C1779DF8011080F820109DF88F
:10169000021080F821109DF8031080F822109DF8A8
:1016A000041080F82310054924208870FFF77AFD84
:1016B0001CBD0000040400006D1B00108C00001015
:1016C00070B5154D2C6B402C00D94024E86AE969AF
:1016D00002198A4202D90C1A04216970214601F0CC
:1016E000DFFD22460D49822001F036FAE86A2044E7
:1016F000E862286B011B0A4829638268A2EB040296
:10170000826005D06978022901D00021017370BD83
:1017100003216970F9E700008C000010140100102B
:10172000CC1B00102DE9F0411D4CA178E06A421855
:10173000E1698A4206D9081AA0700520607002206B
:1017400001F0DAF90021A078164B174DE26A08E0A3
:1017500056186F5C9E5DBE4202D00021A16202E07D
:10176000491C8142F4D31118E162216B0A1A0E4917
:10177000226301F15F018B68A3EB0000886002D057
:101780006078052809D1A06A28B100200873BDE857
:10179000F04100F007B90120F8E7BDE8F081000052
:1017A0008C000010140100106D1B001010B5144CBB
:1017B000A178E06A4218E1698A4206D9081AA07045
:1017C00005206070022001F097F9A178E06A01F02D
:1017D000ADFDA178E06A0844E062206B421A094836
:1017E00022638368A3EB0101816002D0617805293F
:1017F00005D100210173BDE8104000F0D3B810BD41
:101800008C000010CC1B001010B5FFF7B5FC0028B1
:1018100011D0094800210622017042708170C17008
:10182000017141718171C171044908208870BDE85E
:101830001040FFF7B7BC10BD6D1B00108C000010EE
:1018400010B5FFF799FC00280DD00748032101705F
:10185000002141708170C170044904208870BDE886
:101860001040FFF79FBC10BD6D1B00108C000010D6
:10187000114810B5D0F81110027D09BA21F0FF010E
:1018800011430E4A4902D162C18A49BA4902116321
:10189000806888420DD0822001F02EF9022001F0EC
:1018A0002BF9054902201F31087300F07BF8002056
:1018B00010BD012010BD0000AD1B00108C000010F9
:1018C00010B5FFF759FC002816D00C4A0C48116AD5
:1018D000491E0B0E03700B0C43700B0A8370C17012
:1018E00000210171417102238371C1710820907040
:1018F000BDE81040FFF756BC10BD00008C00001082
:101900006D1B001010B5FFF737FC00281AD00E48E9
:1019100000210E4B0170417081700822C2701A6A5A
:10192000140E0471140C4471140A8471C2710222E1
:10193000027241728272C1720C209870BDE8104030
:10194000FFF730BC10BD00006D1B00108C000010B4
:1019500010B5FFF711FC00281FD01048702102229B
:101960000170002141708270C170017141718171FB
:101970000A22C271017241728172C17230220273F5
:10198000012242738173C1730174417404491220AE
:101990008870BDE81040FFF705BC10BD6D1B00103E
:1019A0008C000010064910B5044808600D22822002
:1019B00001F0D2F803490520487010BD5553425339
:1019C000CC1B00108C000010094810B5816839B19B
:1019D000007B000601D5822000E0022001F08CF897
:1019E000034900201F310873BDE81040FFF7DABF3C
:1019F000AD1B0010F0B5FF4800218162C16821F0E5
:101A0000C001C160C16C21F0C00141F08001C1641E
:101A1000F9494FF400228A630B6A23F400230B6216
:101A2000036923F030030361036D43F03003036562
:101A300004238B650B6C43F004030B64436A23F0AF
:101A4000407343F000734362436E23F0407343F0EE
:101A500000734366436A23F0406343F000634362CC
:101A6000436E23F0406343F000634366436823F40E
:101A700040634360436C23F44063436493008B6191
:101A80000C6844F400140C60446824F4401444F4DA
:101A900000144460446C24F4401444F4001444647E
:101AA000046924F00304641C0461046D44F003041D
:101AB0000465046924F00C04241D0461046D44F0E1
:101AC0000C040465C46824F44064C460C46C24F449
:101AD0004064C4648B630B6A43F400130B62C368F5
:101AE00043F44073C360C36C23F4407343F4007346
:101AF000C364C36843F44033C360C36C23F440330E
:101B000043F40033C364C36823F04063C360C36C11
:101B100023F0406343F00063C3649302CB630B6A1A
:101B200043F000530B62C36823F04073C360C36C7F
:101B300023F0407343F00073C3645302CB630B6A1A
:101B400043F080530B62C36823F44003C360C36C4B
:101B500023F44003C36413028B630B6A43F00063F6
:101B60000B62C36823F44013C360C36C23F44013B7
:101B7000C364D3018B630B6A43F080630B62036918
:101B800023F040730361036D23F0407303658314F6
:101B9000CB650B6C23F480530B64036923F0406323
:101BA0000361036D23F0406303659311CB650B6CF8
:101BB00023F400530B64C36823F44043C360C36C35
:101BC00023F44043C3641301CB630B6A23F4000383
:101BD0000B62436823F4403343F480334360436C27
:101BE00023F4403343F400334364436823F4404315
:101BF00043F480434360436C23F4404343F4004385
:101C00004364436823F4402343F480234360436CDC
:101C100023F4402343F400234364C36843F0404368
:101C2000C360C36C23F0404343F00043C364C36804
:101C300043F44053C360C36C23F4405343F4005354
:101C4000C364C36843F44023C360C36C23F44023DC
:101C500043F40023C364036823F0300343F010030C
:101C60000360036C23F0300343F020030364036834
:101C700023F0C00343F040030360036C23F0C00370
:101C80000364036923F4403343F400330361036DB9
:101C900023F4403343F400330365036923F4402302
:101CA00043F400230361036D23F4402303650368B9
:101CB00023F4402343F400230360036C23F4402304
:101CC00043F400230364036823F4403343F40033F4
:101CD0000360036C23F4403343F40033036403686C
:101CE00023F4404343F400430360036C23F4404374
:101CF00043F400430364036823F440630360036C0C
:101D000023F44063036420238B610C6844F02004B7
:101D10000C60046824F440540460046C24F44054BF
:101D2000046440248C610D6845F040050D60056831
:101D300025F440750560056C25F440750564102593
:101D40008D610E6846F010060E60466826F04076FB
:101D500046F080764660466C26F0407646644668DB
:101D600026F4400646F480064660466C26F440069B
:101D70004664066846F00C060660066C26F00C0603
:101D80000664066846F003060660066C26F0030645
:101D90000664066826F440060660066C26F44006D3
:101DA0000664C6148E610F6847F400670F60076809
:101DB00027F440170760076C27F4401707640715DE
:101DC000CF61D1F800C02CF4806CC1F800C0D0F80D
:101DD00010C02CF4400CC0F810C0D0F850C02CF447
:101DE000400CC0F850C0CE650E6C26F400660E6440
:101DF000066903E000C0024000C0092026F44076D6
:101E00000661066D26F4407646F400760665CD65DB
:101E10000D6C45F010050D64056925F440650561FC
:101E2000056D25F4406545F4006505658B650B6C13
:101E300043F020030B64436823F0406343F0806366
:101E40004360436C23F0406343F0006343644368A2
:101E500023F0405343F080534360436C23F04053DE
:101E600043F000534364C36823F0405343F00053EE
:101E7000C360C36C43F04053C364C36923F440237D
:101E8000C361C36D23F4402343F40023C36593016E
:101E9000CB670B6E43F000730B66036923F44013AA
:101EA0000361036D23F440130365CF650B6C23F4CA
:101EB00080630B64436823F0C0034360436C23F0EA
:101EC000C0034364CA610A6822F400220A600269FE
:101ED00022F440520261026D22F4405242F4005258
:101EE00002658C650A6C42F040020A64026842F0A6
:101EF00040420260026C22F040420264426822F0DA
:101F000003024260426C22F00302921C4264A2026D
:101F10008A610A6842F480320A60416841F00C012B
:101F20004160416C21F00C014164416841F0300195
:101F30004160416C21F030014164F0BD10B5FEF705
:101F4000C3FFFEF7EFFF04494FF40052C1E9002040
:101F5000A0F5F420886010BD000000100649302272
:101F6000C1F80822C1F81002D1F800028006FBD5A2
:101F7000D1F814027047000000C000500948062143
:101F8000016107210160002141614162022141603C
:101F9000C168C906FCD400E08168C1684907FBD468
:101FA000002070470000034000B50B46024604E0E5
:101FB000002000F005F802F8010B5B1EF8D200BD0E
:101FC00003498860C868C006FCD488687047000070
:101FD0000000034000B50B46024603E012F8010B77
:101FE000FFF7EEFF5B1EF9D200BD0000F8B5144606
:101FF000074E0A460B19716800258B4200D90A1B4F
:10200000034600943068FFF77BF82846F8BD0000CF
:1020100000000010F8B51446074E0A460B19716807
:1020200000258B4200D90A1B034600943068FFF755
:1020300067F82846F8BD000000000010064802219D
:1020400041600021016741611122C260C163012129
:102050004160002070470000000009404E4810B564
:102060002021C0F8A01100BFD0F8A0114906FBD56F
:102070000321C0F80411494AC0F8A8214FF4806236
:10208000C0F8AC210122C0F80C210B23C0F8843029
:10209000C0F88020AA22C0F88C205523C0F88C30CC
:1020A000D0F888406401FBD5C0F88010C0F88C20BF
:1020B000C0F88C300521C0F808113949C0F8C410A7
:1020C0000021C0F8C811D0F888106FEA11618A07A2
:1020D0003449D0F80C2102F0030207D07AB3012A68
:1020E00044D0022A47D0032A4ED13AE02AB1012A2D
:1020F00013D0022A24D0032A46D1D0F88820D0F861
:102100000431C2F30742DBB2521C5B1C5A43D0F8C5
:102110008830254CC3F30E030EE0D0F88820D0F8A9
:102120000431C2F30742DBB2521C5B1C5A43D0F8A5
:1021300088301E4CC3F30E035B1C634321E010E0A8
:10214000D0F88820D0F80431C2F30742DBB2521C29
:102150005B1C5A43D0F888304FF47A44C3F30E0323
:10216000EAE7D0F80421124BD2B209E0D0F80421FA
:10217000104BD2B204E0D0F804214FF4FA43D2B2AB
:10218000521CB3FBF2F20A60016821F4704141F481
:102190004051016010BD000000C00F40001011034D
:1021A000CE976881D800001000127A0000366E01C8
:1021B00000093D00001BB70010B54FF04021012081
:1021C0000860FEF7F7FC10BD00B5FEF78FF8044974
:1021D0005DF804EB41EA0040891300F015BD0000F2
:1021E0000005400010B502468078FEF77FF80B49E5
:1021F000D1F84432012484402343C1F84432C1F869
:1022000048029088C1F84C02D1F80002C005FBD505
:102210004FF48070C1F8080210BD000000C00050EB
:1022200010B500B101204FF4807444EA0041074822
:1022300000F0EAFC06480321C0F84412D0F800126E
:10224000C905FBD5C0F8084210BD00000005D80044
:1022500000C0005010B5040001D0012000E00020B3
:102260004FF4807141EA0041054800F0CDFC05497A
:102270004FF000700CB1886710BDC86710BD00003A
:102280000005FE0000C0092010B5084CA288402AB5
:1022900000D940228020216800F05EFC21680144C2
:1022A0002160A188081AA08010BD0000F80000106D
:1022B00010B5064C0020216800F028FA216801447E
:1022C0002160A188081AA08010BD0000F80000104D
:1022D0007047000000B5FEF709F804495DF804EB0B
:1022E00041EA0040024900F08FBC000000054000B8
:1022F0000001200000B5FDF7F9FF04495DF804EB8B
:1023000041EA0040891300F07FBC00000005400056
:102310002DE9F0414A4C0027A4F108062178A4F1E8
:102320001C05082864D2DFE800F063046574636369
:10233000868400F0F1FB2078C009FFF7C9FFE08830
:10234000B0802078C0F34111F1BB61780C294BD2E9
:10235000DFE801F006094A0B4A101B1E2026324313
:1023600000F0B6F84EE0002000E0012000F05CFA3A
:1023700050B306E010F01F0F36D1A07840F0800077
:102380002870BDE8F04100F0CDBB00F065F839E001
:1023900000202AE010F01F0F26D129481B381AE030
:1023A00010F01F0F20D100F087FA68B100F0BAFBDF
:1023B000BDE8F041FDF7A1BF00F01F00012813D1D7
:1023C000687808B1207900E00EE0A97888420BD245
:1023D0001B490C39084430601DE000F01F00012843
:1023E00002D100F011FBC3E7802000F085FBB7802D
:1023F000BDE8F081080608D4B0880028F8D0FFF7BF
:1024000057FFB0880028EFD0F2E7BDE8F04100F0B8
:102410008FBB080603D5BDE8F041FFF735BF28782C
:102420000106E5D500F07F002870BDE8F04100F01E
:10243000E7B9802000E00020BDE8F041FFF7C4BE0E
:1024400000010010022803D0032803D1FEF7EEBFDD
:10245000FFF70EB870470000194810B5007810F06B
:102460001F0F1748C07829D115490839012806D00F
:10247000134A0228937806D003281FD112E011488E
:102480000860122012E01048002204E004780CB129
:1024900044882044521C9342F8D1027872B10860FB
:1024A000408803E009481844086000788A8882421E
:1024B00000D98880FFF7E8FE012010BD002010BD84
:1024C00000010010383A00004A3A00006B3A000060
:1024D00070B51D481C4D0078A5F1080510F01F04CB
:1024E0000AD01948A5F11401184B4A780079012C3B
:1024F00006D0022C26D109E01348183828601DE0C8
:1025000002B3897888421DD2002015E000F08F04C4
:10251000200605D504F00F064FF48030B04001E0EE
:102520000120A0400AB922070CD18A68024209D0D2
:10253000C9680142E8D0012018802B60FFF7A4FE93
:10254000012070BD002070BD00010010101D0010A2
:102550002DE9F0412F4DD5F80032C5F808321807A3
:1025600021D52D4800F042FB2C48FFF7F7FCC106AF
:1025700005D500F001F9BDE8F04100F035B981075B
:1025800005D5BDE8F04100F0010000F079B8010781
:1025900009D5400703D5BDE8F04100F0CFBABDE84A
:1025A000F04100F02BB91E4E58074FF001071DD423
:1025B000BDE8F0815FF00004D5F8302207FA04F19D
:1025C0000A4210D06008C5F8381200BFD5F80012D2
:1025D0008906FBD5D5F81412E2070CD056F8201066
:1025E00009B103208847641C202CE5D3D5F83002BC
:1025F0000028DFD1DCE73CB9490705D5316819B1BE
:10260000012088470124D7E756F820100029EAD096
:102610000220E7E700C000500005FE000002FE00B7
:10262000DC3A0000134800B5C16821F0405141F088
:102630000051C160C16C41F04051C1640E491A2083
:102640000860091D0A6830EA0202FBD14FF0E02160
:102650004FF08070C1F88002084B202283F80024DC
:10266000C1F8000100F088F800205DF804EB00F0EC
:10267000C7B8000000C00240F4CF005018E000E0EE
:10268000002802D10149012048707047080100105C
:1026900070B5194C607820B30026184D012810D071
:1026A00002280DD1A8686168401A1549884215D3DF
:1026B0001448406B400011D50120FFF7CBFD667038
:1026C00070BDA8686168401A0F498842F8D300209D
:1026D000FFF7C0FDA86860600220607026700C20C3
:1026E00005E020780028EBD1012020700D20BDE806
:1026F0007040FEF7C5BD0000080100100000094051
:10270000A086010000C0092040420F0000F00F0227
:10271000012370B503EB8203154AC2F8283200BFCB
:10272000D2F820321C05FBD5C3F309030024DD1CBD
:1027300005E000BFD2F8186241F8046B641CB4EBEA
:10274000950FF7D30021C2F8281241F24821C14069
:10275000C9070AD1FDF7CAFD4FF4A06141EA004064
:1027600000F044FA034800F041FA184670BD00003A
:1027700000C000500005F2000D480021C0F84812CA
:102780004021C0F84C120122C0F84822C0F84C1277
:10279000D0F80012C905FBD54FF0FF31C0F8381250
:1027A000C0F83412C0F808120C21C0F804127047A7
:1027B00000C00050044800214FF0011281800170D8
:1027C0004170C0E902217047E400001000B5FDF738
:1027D0008DFD04495DF804EB41EA0040891300F0E7
:1027E00013BA00000005400010B5FFF7E3FF0249EF
:1027F0000020487010BD0000080100107047000064
:1028000030B50749074D41EA00442146284600F00B
:10281000FBF921462846BDE8304000F0F5B900003C
:10282000000180000005D00070B502462148A0F1EB
:102830001C04017811F01F030146498804D0012BC4
:1028400029D0022B27D111E0012924D132B1012056
:1028500000F080F9A08840F0020005E0002000F0C0
:1028600079F9A08820F00200A08021E0007900F032
:102870008F00030605D500F00F034FF480359D400F
:1028800001E00125854063782BB1030703D0A368DD
:102890002B4200D009B1002070BD22B100F02CF90C
:1028A000E068284303E0FFF78FFCE068A843E0609E
:1028B000012070BD000100102DE9F84F504F00209D
:1028C0000090B8784FF000094FF0010A4FF4803BB8
:1028D000A7F11C0600286AD04A4C64E06078022800
:1028E00004D0042840D005285BD140E06179B87855
:1028F000814237D170702079B070414900200C3985
:1029000001F80090401C0428FAD301254FEA06087C
:102910000AFA05F0D8F80810084202D02846FFF756
:10292000D9FCD8F808100BFA05F0084203D045F09E
:102930008000FFF7CFFC6D1C102DE9D34FF0011084
:10294000C8E902090120FFF76BFCE0794006B8F8FE
:10295000040002D540F0010001E020F00100A8F8D9
:1029600004001EE060881DE0E078009019E0009807
:10297000B8B9A07800F08F05280604D505F00F013E
:102980000BFA01F001E00AFA05F0B16801432046B4
:10299000B160FFF727FC2846FFF7ACFC2846FFF79D
:1029A00015FF207804442078002897D11FE086F88E
:1029B000019001245546D846B16805FA04F0084252
:1029C00002D02046FFF786FCB16808FA04F00842FE
:1029D00003D044F08000FFF77DFC641C102CEBD387
:1029E0004FF00110C6E902090020FFF719FCB87882
:1029F0007178884202D10120BDE8F88F0020FBE702
:102A0000000100104A3A00002DE9FC5F384D002714
:102A10003E466878BB46B846002866D0BA46354C74
:102A200005F11C095DE06078022804D0042808D074
:102A3000052854D119E06079697888424FD06088C0
:102A40004EE0A77899F80410E6784FF00008B942F4
:102A500045D199F80200B04241D125484FF0010A12
:102A6000103010F807B0C65539E099F80410B94293
:102A700035D1A17801F08F010191090605D50199A1
:102A800001F00F024FF4803101E0019A01219140E1
:102A9000009199F80200B04213D1A8680843A860D9
:102AA000E968009881432046E960FFF79BFB0198A5
:102AB000FFF720FC0198FFF789FE009948EA01081A
:102AC0000DE05E450BD118EA010F08D1A8688843D4
:102AD000A860E8688843E8600198FFF7FBFB20786E
:102AE0000444207800289ED15046BDE8FC9F000099
:102AF000E40000104A3A000000B5FDF7F7FB044976
:102B00005DF804EB41EA0040024900F07DB80000A6
:102B1000000540000001010001490020FFF7F6BD5B
:102B20000001001000221146802000F015B80000BE
:102B300001490020FFF7EABD101D001003480121E4
:102B40004170034989684160704700000801001026
:102B5000000009407047000070B513460546134C4D
:102B600000F00F00022202EB8000C4F82802C4F833
:102B700024320020DA1C04E051F8046BC4F81C6213
:102B8000401CB0EB920FF7D30020C4F8280228466F
:102B9000FDF7ACFB4FF4A06141EA004000F026F8DD
:102BA000034800F023F8184670BD000000C0005034
:102BB0000005FA00EFF3108010F0010F72B64FF02D
:102BC00080404FF0000202704FF0AA0303724FF0F2
:102BD0005504047202614FF0FF0242604FF003029D
:102BE00002700372047200D162B6FEE7054910223A
:102BF000C1F80822C1F81002D1F80002C006FBD5C6
:102C00007047000000C00050094A1023C2F8083283
:102C1000C2F81002D2F80002C006FBD5C2F8083292
:102C2000C2F81012D2F80002C006FBD570470000AF
:102C300000C0005002E008C8121F08C1002AFAD1E3
:102C400070477047002001E001C1121F002AFBD12C
:102C5000704700000B4910B5486D00050CD40A4AB6
:102C6000906843F698239468241A9C42FBD3486DDD
:102C7000000501D4012010BD0520FEF701FB002056
:102C800010BD000000C0092000000940F0B5054655
:102C90000020034602462B4C4FF4007700E05B1CFB
:102CA000EE5C46B102EB030CA4440CF5805C9CF88E
:102CB00000C8B445F3D0032B3FD302F5C0502044E5
:102CC000037F457FC67F03EB0523857F2D0405EB3E
:102CD00006652B4451EA03052BD021B91A494968EE
:102CE00040318B4225D8194B00215518254405F554
:102CF000805595F800585D54491C0C29F5D3817E08
:102D0000C27E01EB0221027D407D120402EB0060D5
:102D10000C18204600F086FA40F6F57502E000BF78
:102D200000F080FAC11EA942FAD3A0F57061FF3904
:102D300001D00020F0BD2046F0BD2032BA42AFD312
:102D4000F0BD00006D0100108C000010D91B0010B8
:102D500070B50D4CA6680420FEF792FA0B4D02E008
:102D6000FFF778FF48B1A068801BA842F8D308E0BD
:102D7000FFF770FF08B1012070BDA068801BA8425A
:102D8000F6D3002070BD00000000094080841E00C2
:102D90008AB046208DF814004FF000098DF8179086
:102DA00034208DF81500B14A37208DF816001068D0
:102DB000CA464FF6FF031840AD4B40F480701843ED
:102DC0001060AC48AD49B04DC0F80090AA4800680A
:102DD000A0F56C50FF380860A94900F5E050086084
:102DE000A849400A0860F8202870FF206870A87081
:102DF000FDF7F2FAA64CA54A002094F9051052F806
:102E000021102B1803F580530A5C401C83F800281E
:102E10006028F6D34FF4E175294640F24910FDF7DA
:102E200019FF294640F29F10FDF714FF4FF4005B95
:102E3000DFF860825D46207808B1FFF729FCA079B1
:102E400028B1012819D0207800286ED0FDE00A2092
:102E5000FEF716FAFDF760FF18B100BFFEF7C0F9E4
:102E6000E9E70120A0715D4684F803A00620FEF783
:102E700007FA0A20FEF704FADDE7192229468548F9
:102E8000FEF7CBFA98F8180000287CD098F80000DC
:102E9000062873D2DFE800F072030B46464A40F280
:102EA000044000880390D8F80410814266D098F856
:102EB00009104FF00109404601295FD1D0F80A10EE
:102EC00019B975498969C0F80A100026804617E0CB
:102ED0000720FEF7D5F9D7F80E00B846871B402F1C
:102EE00000D94027A9193A466C481931FEF795FADE
:102EF000D8F80A003A463044684900F0D5FA3E4412
:102F0000D8F80E004746B042E2D83978012935D1C9
:102F10004FF0E0220906C2F88011D7F80A0000F04D
:102F2000DDF82BE04FF001092BE087E098F809105D
:102F30004FF00109032924D14F49594A00260B6853
:102F4000136016E00720FEF79BF9D7F80E00871BE9
:102F5000402F00D94027A9193A4650481931FEF7A9
:102F60005CFA45483A46006881194C48FFF73EF83C
:102F70003E44D8F80E004746B042E3D898F818000F
:102F800008B1464600E01CE098F80800C00613D5DA
:102F90004349012203A8C1F800B005F11801CDF89A
:102FA0000CA0FFF737F8307820B1C8214FF47A70C1
:102FB000FDF750FE307E20B1307A800701D5FFF753
:102FC000F9FDD8F80E001B3505443248FEF738F9F4
:102FD00030B302203349A0715D4681F800A00B2078
:102FE000FEF74EF9B9F1000F1AD02F484FF0000943
:102FF000816842F2107283685B1A9342FBD34FF4EC
:103000002F714FF47A70FDF725FE2848406D40057A
:1030100002D50020099001E0099808B9FFF7CAFD20
:10302000E078401CC0B2E0700C2802D30120A070F0
:1030300014E7A07800283FF413AF0FE701202070B9
:10304000FFF7F0FA0120FFF705F91648007800288D
:10305000F1D0002105A8FFF719FE0028EBD084F875
:1030600006A05D4684F803A0E5E600000CED00E054
:103070000000FA05C000001008000010B0000010A9
:10308000A8000010AC0000106D01001074000010CA
:103090000C00001054010010483900001401001009
:1030A000000000107C0000100000094000C0092052
:1030B000084A34231360C2E9010107484FF47A71CA
:1030C0000068B0FBF1F0D06002F11401104600F08E
:1030D00033B80000E81B0010D800001072B6034996
:1030E000034A01401160FCF7FBBF000080FFFF1F97
:1030F00008ED00E010B572B606240E4951F8242000
:10310000824212D90B49783951F82410814207D1F3
:103110002146084600F0AEF821460846FFF7C8FFF2
:103120002146084600F0A6F802E0641C1D2CE5D9F3
:1031300062B610BDC0390000004A1047F11FFF1FE2
:10314000324C0026FF202660A680A6716071FEF733
:1031500085FFFEF74FFCFEF771FFFEF733F9002005
:10316000FEF78EF8FEF70AFFFFF774FD20B3042088
:10317000FEF786F8264F786D264D000514D4FFF72C
:10318000E7FDC8B1FFF7E4FDB0B1FFF7E1FD98B18D
:103190000420FEF775F8A8681F497A6D120503D45C
:1031A000AA68121A8A42F8D3A86842F21071AA6873
:1031B000121A8A42FBD36671FEF7C0FEFDF7ACFD22
:1031C00080B100F043F968B10220FEF759F894F994
:1031D0000500401C03D111488069FFF77FFF0120E3
:1031E000607004E00220FEF74BF866706671FFF72E
:1031F00031FD40B140210A48FCF7A7FF4022D10130
:103200000748FEF7F3FEFFF7C3FD00000C000010B7
:1032100000C009200000094080841E0048390000D9
:1032200014010010FFB50246002002EB42050146E2
:103230004FF440566C4603AA6B1844F82130B34251
:1032400002DD002004B0F0BD094F07EB6307DB0788
:103250003F78575401D03B095354535C8F0003F01F
:103260000F035354BB40491C18440329E4DBE9E72E
:103270006D010010084A32231360C2E901010748BA
:103280004FF47A710068B0FBF1F0D06002F11401E4
:103290001046FFF751BF0000E81B0010D8000010D7
:1032A0002DE9F0471D4A00234FF40077156A4FF4CB
:1032B000FF79C5F30724DFF868A04FF4E05CDFF87E
:1032C0006480194E25E0B84216D213280CD0142879
:1032D0000CD048450CD0A0F58072FF3A0AD03E28A9
:1032E00013D81AF8002011E0EAB20FE022460DE0F0
:1032F00055220BE0AA2209E0604506D208EB000245
:10330000A2F5805292F8002E00E00022F254401CF8
:103310005B1C8B42D7D3BDE8F08700008C00001007
:10332000083900006D0100101401001070B50D4641
:103330002C49496D490521D4B0F5007F1ED32A4997
:103340002A4CB0F5E05F1AD28A68A369D21A284BDA
:103350009A4204D38968A1610021616061612549B5
:103360000023A1F5D05207E0C4181444CE5CA4F5A4
:1033700080545B1C84F8006EAB42F5D370BD62696B
:1033800022B98A68A2618A686261A0601A4A527989
:10339000002AF3D18A686369D21A184B9A421BD269
:1033A000174B01221A708A68A26189686161A1685D
:1033B000401A6168884203D9616A884200D260601D
:1033C0000620FDF75DFF61682A46BDE870400948A8
:1033D00001F50051FEF70ABEBDE870400C20FDF774
:1033E0004FBF000000C00920000009408C00001001
:1033F000A08601006D1B00100C00001020A107002A
:103400007C000010FFB50DA60446E1CE8DE8E1007A
:10341000022902DA002004B0F0BD6018002100F893
:10342000011D6946B3FBF2F502FB1535B3FBF2F360
:103430004D5D00F8015DA042F4D8ECE73031323345
:1034400034353637383941424344454646F2044024
:1034500000210088A0F51942993A0AD04FF4C040E3
:103460004FF4002208C890421944FBD309B1002050
:10347000704701207047000010B572B63324084B26
:1034800010C307C307484FF47A710068B0FBF1F02E
:103490001860191D0248FFF74FFE62B610BD00000C
:1034A000E81B0010D80000102DE9F041144C2368EF
:1034B00003B920600020134D636803E00F5C1E1801
:1034C000401CAF559042F9D398184FF48076606055
:1034D000B04212D12068FFF70DFE0A4D143D286856
:1034E00000B1FEE7324607492068FFF7C5FF2868AC
:1034F00000B1FEE70020606020600020BDE8F081A0
:10350000C4000010101C001000050F0A1B1E14112F
:1035100033363C39282D272263666C69787D7772B3
:1035200050555F5A4B4E4441C3C6CCC9D8DDD7D2A3
:10353000F0F5FFFAEBEEE4E1A0A5AFAABBBEB4B193
:1035400093969C99888D878283868C89989D979283
:10355000B0B5BFBAABAEA4A1E0E5EFEAFBFEF4F173
:10356000D3D6DCD9C8CDC7C240454F4A5B5E545163
:1035700073767C79686D676223262C29383D373253
:1035800010151F1A0B0E040103060C09181D171243
:1035900030353F3A2B2E242160656F6A7B7E747133
:1035A00053565C59484D4742C0C5CFCADBDED4D123
:1035B000F3F6FCF9E8EDE7E2A3A6ACA9B8BDB7B213
:1035C00090959F9A8B8E848180858F8A9B9E949103
:1035D000B3B6BCB9A8ADA7A2E3E6ECE9F8FDF7F2F3
:1035E000D0D5DFDACBCEC4C143464C49585D5752E3
:1035F00070757F7A6B6E646120252F2A3B3E3431D3
:1036000013161C19080D0702000021104220633018
:103610008440A550C660E770088129914AA16BB12A
:103620008CC1ADD1CEE1EFF13112100273325222D2
:10363000B5529442F772D662399318837BB35AA37A
:10364000BDD39CC3FFF3DEE36224433420040114A2
:10365000E664C774A44485546AA54BB528850995CA
:10366000EEE5CFF5ACC58DD5533672261116300672
:10367000D776F6669556B4465BB77AA7199738871A
:10368000DFF7FEE79DD7BCC7C448E5588668A77832
:103690004008611802282338CCC9EDD98EE9AFF96A
:1036A000488969990AA92BB9F55AD44AB77A966A12
:1036B000711A500A333A122AFDDBDCCBBFFB9EEBBA
:1036C000799B588B3BBB1AABA66C877CE44CC55CE2
:1036D000222C033C600C411CAEED8FFDECCDCDDD0A
:1036E0002AAD0BBD688D499D977EB66ED55EF44EB2
:1036F000133E322E511E700E9FFFBEEFDDDFFCCF5A
:103700001BBF3AAF599F788F8891A981CAB1EBA1AD
:103710000CD12DC14EF16FE18010A100C230E32029
:103720000450254046706760B9839893FBA3DAB3D1
:103730003DC31CD37FE35EF3B1029012F322D23279
:103740003542145277625672EAB5CBA5A8958985A1
:103750006EF54FE52CD50DC5E234C324A0148104C9
:103760006674476424540544DBA7FAB79987B89771
:103770005FE77EF71DC73CD7D326F2369106B01619
:1037800057667676154634564CD96DC90EF92FE931
:10379000C899E9898AB9ABA9445865480678276869
:1037A000C018E1088238A3287DCB5CDB3FEB1EFB11
:1037B000F98BD89BBBAB9ABB754A545A376A167AB9
:1037C000F10AD01AB32A923A2EFD0FED6CDD4DCDE1
:1037D000AABD8BADE89DC98D267C076C645C454C09
:1037E000A23C832CE01CC10C1FEF3EFF5DCF7CDFB1
:1037F0009BAFBABFD98FF89F176E367E554E745E59
:10380000932EB23ED10EF01E005EBCE2613FDD831E
:10381000C29C7E20A3FD1F419DC3217FFCA2401EB0
:103820005F01E3BD3E6082DC237D9FC1421CFEA0A0
:10383000E1BF5D0380DE3C62BEE0025CDF81633D90
:103840007C22C09E1D43A1FF4618FAA427799BC580
:1038500084DA3866E5BB5907DB856739BAE4065870
:103860001947A5FB7826C49A653BD987045AB8E660
:10387000A7F91B45C6987A24F8A6441A99C7257B50
:103880003A6486D85B05E7B98CD2306EEDB3510F40
:103890004E10F2AC2F7193CD114FADF3702ECC9230
:1038A000D38D6F31B2EC0E50AFF1134DCE90722C20
:1038B0006D33D18F0C52B0EE326C8ED0530DEFB110
:1038C000F0AE4C1291CF2D73CA947628ABF5174900
:1038D0000856B4EA6937D58B5709EBB536688AD4F0
:1038E00095CB2977F4AA4816E9B7550B88D6346AE0
:1038F0002B7597C94A14F6A8742AC896154BA9F7D0
:10390000B6E80A54D7896B35EB3C904D53444F537E
:10391000352E3000020201000110000004F80C00F6
:10392000010001000000000000000000000029EF7D
:10393000BEADDE41544F4C20465072696E74464114
:103940005431322020200000000000000010000050
:103950000020000000300000004000000050000087
:103960000060000000700000008000000090000077
:1039700000A0000000B0000000C0000000D0000067
:1039800000E0000000F000000000010000800100E5
:10399000000002000080020000000300008003001D
:1039A0000000040000800400000005000080050005
:1039B00000000600008006000000070000800700ED
:1039C000FF0F0000FF1F0000FF2F0000FF3F00005F
:1039D000FF4F0000FF5F0000FF6F0000FF7F00004F
:1039E000FF8F0000FF9F0000FFAF0000FFBF00003F
:1039F000FFCF0000FFDF0000FFEF0000FFFF00002F
:103A0000FF7F0100FFFF0100FF7F0200FFFF0200B8
:103A1000FF7F0300FFFF0300FF7F0400FFFF0400A0
:103A2000FF7F0500FFFF0500FF7F0600FFFF060088
:103A3000FF7F0700FFFF0700120110010000004098
:103A400051C20313000104204801090220000101B2
:103A50000080320904000002080650620705820255
:103A60004000000705020240000000040309041C96
:103A700003410054004F004C002000200020002093
:103A800000200020002000200020002803460050D5
:103A900000720069006E007400200046006C006136
:103AA000007300680020002000200020002000207B
:103AB0000020001A034600690072006D0077006163
:103AC000007200650030003000300030000E034D01
:103AD0000065006D006F0072007900001123000086
:103AE000000000004524000000000000000000006D
:103AF00000000000000000000000000000000000C6
:103B000000000000000000000000000000000000B5
:103B1000000000000000000000000000C794809A30
:103B2000E9020000E90200004D10000071100000E1
:103B30004D100000711000007110000071100000A5
:103B4000291000009B0200009502000009040000FB
:103B50000103000051060000C9020000C902000074
:103B60008107000029100000000000000000000094
:103B70000000000000000000000000000000000045
:103B8000000000000000000000000000AC3B00004E
:103B90000000001014010000342C0000C03C0000A4
:103BA000140100103C2C0000442C00000000000018
:103BB00000000000000000000000000000000041C4
:103BC000544F4C20465072696E742800000000006B
:103BD0000000000000D4284B3D0000000000000061
:103BE00000000000000000000000000000000000D5
:103BF00000000000000000000000000000000000C5
:103C000000000000000000000000000000000000B4
:103C100000000000000000000000000000000000A4
:103C20001300001000000000000000000000000071
:103C30000000000000000000000000000000000084
:103C40000000000000000000000000000000000074
:103C50000000000000000000000000000000000064
:103C60000000000000000000000000000000000054
:103C70000000000000000000000000000000000044
:103C80000000000000093D000000000000000000EE
:103C90000000000000000000000000000000000024
:103CA0000000000000000000000000000000000014
:103CB0000000000000000000000000000000000004
:103CC000C1BBCD59DF6DD8681FEDE9CD639D7B4B3E
:103CD000078210F088E3DB7C9DB51A3E38DBBD9B84
:103CE0006AE504DD69779615287D64EB34B96FE7E2
:103CF0001508A526801BC7CD86F0AD368D7D6CC01E
:103D00003C96819BAC132F404B8611BED62EC7F834
:103D10007E5268BCB52C20905435D8B909A3FF75E4
:103D2000258F8AFEAAFFBC8FE941A3311725CCD588
:103D3000CEC8C2177528A616F4D3F8D9BE2CFFD862
:103D400072A382ED7B7525D30CB53A5047909DAF99
:103D500089A1C6AB5F0D08BBB70FD560AEFD98C398
:103D600031D846A1E446D313E23B43D5126DACA44F
:103D7000EB89B83C6E9B728721D614432169AEDA79
:103D8000B67ED9E9039CA775016D440D70CB1976F9
:103D90008EED246259C8E1B142A59CE5689E239C42
:103DA0004FC4BCECF5DAF2B1F6A94DDCC31AD08DE4
:103DB000E344FE8C7AAF4D26E6BD2B92DDAA755406
:103DC0004F800E29F7184343903729EFBE1BBC7D67
:103DD000BCFCD5485CD79F516C8429A454F0568A0A
:103DE0000612A8DF5787CC5EBD6585920D1115CCF4
:103DF000DC152CCF8001EEED32D56719D008E5FD3A
:103E0000931EC000C6E6CE0174561700A24D9598C9
:103E100013CC684E8E927FACC0003571DD3C00370C
:103E20008E372479455BDC2CE95F6F3E0D3301D280
:103E3000DBD409145CA71BB33D9C52B4ACBF752DF9
:103E4000DC06B5C192EB948D7B16959E543FE54BF5
:103E5000F28DEB856E15D4F11ED02BB26B97E9492C
:103E60007FF00932A3D6205BF6B10D2CB2C179B533
:103E700073136EB3AB0CB5450CC6738788CA337524
:103E800011760A08E01B807D763E513E03EA354CF0
:103E90005DF79DB25F7CF5E6BD3AF084869E83288F
:103EA000CF869D2CC81244B3C122D0F9630457E7D2
:103EB000A54308BA6BECECD52DA5565FE523055458
:103EC0001116E44F70412F95D65912125AFBB24683
:103ED000E171A5F3A496FC9EB1612C721E3B803368
:103EE00086BD253522695E9F445BDE08BFDE4D211D
:103EF00057785B7C788D9295A006E15C4E69FD7FDA
:103F000003B4487579C1EA4E12BA2704CCA77B25C1
:103F10004BA14893B2B70038BD6B4B335AD68B6F69
:103F20001E41A0F972EAE4B9CAE439D3D2A611B7A6
:103F3000A50CD6C525A468CDABF19F8FF15FB7D591
:103F40002721418F34176F7803F1777266C3F760CA
:103F50007959821DE19C4E70E71FF7B8DF1982F393
:103F6000565D7C68D303BAA91DED365FB7A7E7C6D7
:103F7000DC80B6C7EDBD370D2AD7A7087F4C9A1253
:103F8000FE43328C2FAD39BDE2083418C16EE0E03B
:103F9000D25252DDFC7F8576960918F4E9573E111E
:103FA000B26633CF72514A81E0A364082CAE82E03E
:103FB000799545B3AC32C521AF67C5402D603BB59F
:103FC000D8ADDDF7C9651A2AC6506D120B253D0420
:103FD0006DAE8F972FD48C63867A7D85D302D7FF01
:103FE0007100EFEE62C77E02C33CBAC4D3CABF2DD4
:103FF0004B15A142F41DDD6DFCDC16CDF9212EFE22
:10400000DC1040A40C19492861C12A904078D413CF
:1040100007C8C1D65EDB1C0BD1C4C0372A6C4A2648
:1040200030FB0C9E5170EF8962F2F6E8758D7D27AA
:10403000BB33317AEE7D0D6C74330A6DDF7A45D473
:10404000B0F9AEF8386481226D177B981F3397F270
:10405000F14BFA327CA3AC7F6FD0CE6967BA375E82
:104060004516B13272834A44D60410F3B8F70D28CE
:104070007987A700C0FA503BEA5C701A5344003BB2
:10408000DF1EAA64C4BA4DE9B5CE4D610CEB97139F
:10409000B469F797AE42DACF63486CF24FAB8298BF
:1040A000ED1252F8A0EA74C50076F05C5464058302
:1040B000395C7F34F3FAD1E663140D8A855D82DDC5
:1040C000B924B500BB69D614AED49876E008AAB876
:1040D0003C50A559EA6575C323F3D13C2E0FBD3D75
:1040E000CAD6D8679CEFB0B02F4CD6B1E653EBEEF2
:1040F000C774492177CBF18C2DA00E7F8D6DA793CE
:10410000000701EBE6EAA3825CD716B8D382426CC3
:10411000D29B0E580932F20D18C85C812F091C7B06
:104120007A04FC65FFE53B6387632D3C7365C0073C
:1041300035F270407B94666C032645562C29E8BB0B
:1041400063606B72F1E034AB990D864083DDDA9CDD
:10415000EB5777217F9A187D957503A05012E1E403
:10416000027909B6BF2F1B68125B0C2F1DF3274283
:104170006A077D76614138404704A8BF711AAFFDD8
:104180008EE98DDB229D395E09568231A94D709FE3
:1041900017EA3990040EF11799CC5AF944BC35F955
:1041A0007AE69D0ECAE55C9230D0675C462BAC2A5D
:1041B00058014E365CFB8400B90884D3842D9D01E0
:1041C000A03EF743FBA4747B80C03FEF1214BA2BD0
:1041D000E78EC8A2AC869856F63EB6325814A8B3FD
:1041E000E215FB5C80E66CC3BD3E595D9D5AD61955
:1041F00040A509623C770E9DF7EB1EDFADE62AEB8A
:104200002BFB5423DAE6B44FE0277ADBFD13D7BC4F
:10421000EF8887257A0C273A91AB59BCDD9BC7EE16
:104220007B41A984B9573AF51EF4C05E9DD98D1D16
:104230002CA1B9BF77757BB62E13E83F8D57A7C762
:10424000DE629D82CCF74E1113363D3AAF00047EFC
:10425000B9AC3A674CD01B3FE4D7F527561913CABF
:104260000B58D3CE436569677F23FD91D451B8D1F4
:104270008AD3C87E311A6140C38C5BE833AAFDE45F
:10428000122B761D75E9A36ED011C78F30DAD935A0
:104290007E830586E035F59CE10D9E9385E422DA68
:1042A00065FFA2A98698DCBB3F68B787DCAE4C09E6
:1042B000516554E9196E4AFBF630B514940C464A20
:1042C00097C39B79C85500DEFE7BEFCFE42F3DB34B
:1042D000BFA16A0BD3FD3F16AB0E2E94F6B0FAAA1F
:1042E0009C9F46FC49885BCCD00B3CC012ECB04193
:1042F000D2991D4390B141A61E492034214019E7AF
:10430000CCD36C7B74C4A60480E4F4346A73345D4B
:1043100061E677276888850426B9DD6AE334DB45E2
:10432000AF369D048E127DFBCA735B4838A34105EE
:10433000693B991294F399D3AA71D60EF0010C1F20
:1043400065EA07668B8B580F5826EDC549556D8772
:104350003A258A1ADF7114EE63DE10C4E4A76FE613
:1043600069A101DF891625962ED884E62C669E9FCA
:104370008E615110F1E2BCA0960DC522158F698C9B
:10438000A6236EEB22ED0ECC1B3FA45EC8D77B1C90
:104390009FAAD7E60B0F33DC9EF13253A79E9B4CAE
:1043A0003CBFF341015B6D945813831D8B65B1B025
:1043B000196A7900985B2DCE1472DBBC3ABB5308A6
:1043C0003407B14342334C713939EB2DFFDBDC2B21
:1043D0004E09A8CAA4C68B44AAA74339DD13CA1044
:1043E00032D3B8D313AC258CCB4C15EECB5046133F
:1043F00004EF821045AF66A808E013585D88D974B1
:1044000006421C70EFAAFE4A1C4BA4B0C36EADF767
:10441000C5DFC47AE696A03552B8C81D5742704C25
:1044200031CFECE9B790A14518C15E45A15F444288
:10443000C31D2774D94381B609128CB3249270ED41
:10444000C1CF151956A5E38E29AF638C27020EC381
:10445000FB324858740F7925A508BE4DF4085FFB60
:104460008A39303CB1006E401AF4543B9091F9B552
:104470006A0179862C532CE4D48C1CD3BDC8B78D2B
:10448000774E11977CE1EADE565A801B5DD87CE0BE
:10449000A4A9669FD63EEF196E29CAACC94973A07C
:1044A000FD052A116B3CAC671C931DCFA63670E14D
:1044B00007B49900C46134A310549868A858F564EF
:1044C0003B0F8A2BE39C992EB0D8C159D5B888E40C
:1044D000F9D6620B166CADEE7596A352E94E9B179A
:1044E000D9A2DCDC20014C4288AA135A36BC52887F
:1044F000E8434B6D7B6AE91DF6463C99DA9AD8840D
:10450000C03DEDB744827EAC63907161EE3150AE38
:1045100024DCB2BFCD9E476287A775DAF9835F1CA2
:10452000E0F23E262D5D98B2126996E52C1E9AB5F2
:1045300007B957BB7D432E102D745E5D9CB1C5EF4E
:104540003539D1E12D76EE48F36171A2A58CBAE937
:10455000E154C7C080ADBB84A460CE791A03EE716C
:10456000B4F8C5F7F7916BB1BC9F6E8E1E9AD7FE5B
:1045700088571B42FA2A7B3CEE568D6C216AC0A2FA
:1045800011F9A903BDD78D48D8504158C141E678EB
:104590006782910FB25128C96A3743CA22006C0F53
:1045A00095D00F1186055AC0EC43CD79E4BA8096B8
:1045B0003B7889B8DB04A4E65593FBCB57DDCA51A1
:1045C00062FFD60563EB9BDF92EF7D48C3DB39D7F3
:1045D0004FB1CF7C49DD30752F6550E9FB4E35BAC0
:1045E000C0472ECB34903566C38D68E467FE4E2AF3
:1045F0000712D4EABD891BF7539A57ADBDD0724B51
:104600004A6064860971FBC0DD2796C1D349734CAB
:104610005DE1DF2256E2687F7523002937268E0B85
:10462000BFAFD5EE0B51B31D4DC596108B160E0CBA
:10463000CF0F992252DA706F1888396088B993BA0F
:1046400093BB67345FCFB1B4E41D94BD84B5B404AB
:104650007322DA7A2AABCAB1E698ADF909DF29E903
:104660004211EB8C188E5AE03E0FC5679D2B0484D7
:10467000A410D84819FF76823AB3BBA4E3D3B71B82
:10468000DE0B262C38D4D37392383A2C6F79D92F7D
:104690001E88BFC74770063A104F35CFEAE2F09246
:1046A000CF480CF116EA0544DB0414E067AB979F92
:1046B000E8F911F3B1EE1FFC3F4F670D044D65475C
:1046C000E014DC46EB309578B4596DDEFA01A87F32
:1046D000FEE1F7DCF8D4718BBFC8356FAEEF6F65C4
:1046E0007910EB1956CE8BC0CE45DCDF0D791392D5
:1046F0005CF88D437E39C36D457FC298DF2A3799B8
:1047000042EF97C7B1F33069C5A146C4AB25E72C8A
:104710004CF75C7CD3D6F8A0549A23056CF47CBD8E
:10472000579B51DEECD137DDCF862E0F1332DFBD24
:1047300055E6C375453B1992CC1DAF7C7FB7BAFDDA
:10474000EC2DB6A24438FA1BE000244EA2FEE33C56
:1047500093DD31FFFBA2C00158DAB4579CC0884EEC
:1047600046048DEB90BD442B6D43D79F6C2362B103
:10477000C65C5B05B863138582DA3A59BBDB3382CA
:10478000D6D685C9132D3B7F828BC3D74934EA4ED9
:10479000290C74899B5F88C120FF65CC72E151941C
:1047A000C34E4F05358C342F3A297D7F8CC53AF89E
:1047B0008B074E1D75311330EB5DF6661E62741B60
:1047C000B671F37A296A9A0EA6241AEAF655453C80
:1047D000C62F4919AFFD9FFFBCE1B279553C85FC5E
:1047E000AC8C63AF8C1EBAA5894F62D5ACE53C4654
:1047F000CF800FA39EEB82219798256A35E25DE971
:1048000070337EC559B161733D4CC04E95B9BC56ED
:104810007681FFE5913110B86E7498D3DB6080E942
:10482000980401CD3458D24BDEC1BD0336318AA580
:104830004D863F33E96B9697995AF149DC818C9804
:10484000C6692F12E52D2C0EFC3BC790FF38228E37
:1048500011247E5DECBF8E05C4721E7D2254F4D2FD
:1048600078B7AD8C9B20BF3FE44C22DFCEA4CE1B9B
:10487000FD08035E8B09E7F0857B82C1CBF78B37A0
:104880005B91C349A0C18FF0A9F44748D24ACA49F5
:10489000E4E15ACA5A4E32BFED1BA43E50B1661C29
:1048A0008C17860E417D6BA023E2C409F1D2F6136A
:1048B00034CFD4B67BD1822BFD83F9F00A29496D20
:1048C0003ED43B1DEB917844C00BF913A2EB782842
:1048D000D702AA884B939F19236AE85408388F8E11
:1048E000BE7B6F3C4DB76DCB64DCD2BEF0E202867E
:1048F000142EE8F861DD6B0CC876B07F99E9115091
:1049000094675A03C7F83983F7B1BAD497ACAB2987
:10491000E9B434C1EF4F976C13D0B0C1B5F5A7AA75
:104920001C3DDDAE6EFFBEDF9A9E1CF049E564A61D
:10493000A4442197851A9701784423DEAD08896D38
:1049400069665A0E8D59CB3687E8EE1CC368E08342
:1049500072A1B7D567BD7943DDC5BBF0933D924BDE
:10496000BC3B5F9D3A8A7A619B30AE240BB094B811
:10497000EFAF322424405D4C3809BA77F9EA61760A
:1049800025524F755493AF463DBE324812F25085C2
:10499000DE43C4F84DDF86D2C84FF8B646BB9ED47E
:1049A000B8EE069B1E0C86CA0E4203175EEB079FED
:1049B0002302EA62CA8F071538994041338ADFE63D
:1049C00048577A38396A132B1AB3DD467014DE2241
:1049D00031B39F5DF667D22FA9DE4E00A98130C1A9
:1049E0000EAC743FEF7F5CF23A224862E15ACE523D
:1049F000B663762E9AC2DB61E798358A6FF5A29F7F
:104A00005B0192D0E8EE950770EE5AA0D495304B3A
:104A1000D24E582AB371222D78F55BAA2A480C1180
:104A20001EF146C1B37AADD5E169F8912C8E1C0C0C
:104A30000CA3AA0727D7A126B59C4BA26CBDDBDA35
:104A4000D0C3FD29F6D4C269A212F95962A5523920
:104A5000B1DBF37D71E836F75E5BC52BC13FBE7DF0
:104A60008C0ED0312E47F1FF8683235407654E13F9
:104A70003E05C4FBB633C240535BF616FCAA8288DF
:104A800016B790AE8A61BF651B17EF126594CDC053
:104A9000350253CC3107ADCC84786ADAF2CD98D3A5
:104AA000F9BF3A1794F094899E51EFD753BAF68F15
:104AB000EB39035C06CE26860E60A000F93D38AACD
:104AC000968474E68C100C2B3E0BFD02F79D3EB6CF
:104AD000AFB96FCE0A44B4242464E59B40785D21CD
:104AE000C91ED3E7E4579C0DD52F63B8FA57CC6B9A
:104AF000D23BF9CFDFF88826E88325888F98A27FFC
:104B0000ADBE39C00842A40E89EE71A546EB6FE731
:104B10006A8CEA47E8A94EA6DA4544D5D5AE938813
:104B200015E38275C5B055EC6AC4592E941C760104
:104B30007E45CB9777D9A32C23F7E5D0587A5950E7
:104B4000AADCF2AFA1BDC6C38ACAA7E9BC50E7D5AB
:104B500015B178988E080412F87AA0CDEB356B2E3B
:104B600036C765383142E31DED38674350C5BFA6EF
:104B7000B573DDD15B2F91607C1F26E0BC203F43E5
:104B80004418F1CD965375B31B3D3B073B8E946D96
:104B9000E2CD94DAC7DCD839E1D1EE33FD3E2BFF0C
:104BA000DAE46FF1FD56867921F3D1AE810BEC1575
:104BB0002E14301FF46C76BAB5FADD64D9C029889A
:104BC000D9E0D722EF7AF047308733A70999F4E785
:104BD000B3BB220EDF04E4B1DD36BFBBFECD4B36E6
:104BE0006A1C3B67FBB1D00373F9E2B4DAEA53EA1B
:104BF0002C0E1842AA496FB2EC35F22BA755AB70B8
:104C00007B9DC169A7F52F19CA163547BD1F032A19
:104C10001F25503EBD04489DD75341051EB1D78F77
:104C20005A40A5CCDF6049084A8B6E74D48DA15BD5
:104C3000142DA42EDBFA278B725E67AF4E355D858F
:104C40008F94C4F2D79E7EA310089CD805DA071E65
:104C5000AFF47E99C3F6A6BF623C800E920CFA6256
:104C6000D48E784F5E8BC0DBEE1888FD983486B604
:104C70009F18346964EA244B6C9C0C7C2C81573B54
:104C8000D90BAC62773365E6A3A99B139639E5216E
:104C9000A697CBEA5DF3E0D382F5A85C72EB7513BF
:104CA000C1DD5E88AFFF48C73ACFDEA49E4ED582F5
:104CB000FB8983E753AB52B4051D50650DB35DB658
:104CC00036D12D170F8D3865774E10E0875AD642B2
:104CD000689E5021CE259E5C6E055BF90C23962EB6
:104CE00022FCE991DF335254D6755195C153CE74ED
:104CF0009D7B698E0A3AD1F423A0E4CEEB961A2666
:104D0000AFE6B49F9B83ECDD803DF87D42F76C718C
:104D1000D691F12E422BCA2D5CCEF9D58A2F4F0D9C
:104D20009AFB730196FF26CCD5C4637188107AE094
:104D30002C72377D379489DB354560BF507CBE2FA0
:104D4000B36CA82F5AF74C730F9102DF757A42C3E8
:104D5000DBE996848FDDBA7247FBDA9770931A7697
:104D6000880CAC38ACAA95846779B86BE850410AD6
:104D70004ED2E2A0275ED2B1A8E55E64052BA2BCAC
:104D8000EDD9D5064B6CA4213CFD032C2740829025
:104D9000BE4A38B30F20D9873625BCC4341272BC42
:104DA000209F3B506C0ECA52C8734C266B77B35889
:104DB000F96E9E6AC1C5CA0FEC625CDEE736F9592E
:104DC000BC407D8ADE114AFDAF5632A7445E7B5B54
:104DD000B5E32860C0995399E714AC16777E5D4B14
:104DE0005EDE191DEDB8C96FAD6FEB0835979159AF
:104DF000EF48B340372C609D64F7B8DDB8A69F69D3
:104E000019887950ED67BDC2DAFC61529589E2BC20
:104E1000D85B8EA5E1BBE9D2586740C7E0F99B5447
:104E2000361758CADBFCAB8CD67E57107EEF6C9CD5
:104E30001E4812954F4D85A36791132A83FBBFED42
:104E4000BC6C81E77FA91D14389A1A1BBEC2EC6B9B
:104E50001C5DC6276A34E55A8FECB1B44C11A867C3
:104E60007E358C0D213A9C83360E4A237622D1362C
:104E7000DD3A6D768D7832E52D31CE576FD66147AC
:104E80009D97E08C8A32FB3D6F3C362BD589D9EA61
:104E900018AAD7E2E36810B6E6078B3412D56E2D58
:104EA0000EC574100393A60E4157AE5018CBC6B76B
:104EB000CA8C65DFEC245F43F62C771C25FF2DDBC5
:104EC000949A35341CFBD3CC75F6EB57E3114EEDB9
:104ED0001F7682EB9F43B19ACA9E3FA80CAFC9A62A
:104EE000BC1A879A7503DC4B9C4E490091A2F628A8
:104EF000DCE1A8DF768645BAE17A960C0F8AB60324
:104F0000FB2A71BEC9D9F413DFF54FDE621F1ABF49
:104F1000DF3B107D398266177C2BFB652DB2FA9141
:104F2000D8060E6AEE08F47B45CC430FDA5CE72521
:104F300097176C700C990C7A5DC2E8B332D0EB3ED7
:104F400016E83ED602F3030495ED61B0076308BE90
:104F5000798F6926590FA1281BD7A9D35DAFF227F6
:104F60009E32610956BAE203A6F287C669DA58B2E0
:104F7000148F1AC1471D955FC3D966A39844D50BFA
:104F80004FF660DADB4562B8416897901083E9E834
:104F9000FDB8F04D7986709D72346ACEE71418031F
:104FA00007F8ABEE21E61DAE99C8576242EA094206
:104FB000002EC8F5B81FA8AA3B5676AB1957EEE6E7
:104FC00069D45998D61DCCDD1A36618C32CD41A3F7
:104FD000DAE029EA31C0932776DDBB0998D5402471
:104FE000379836260D3297256F83D8B76B564C6AA3
:104FF00016BEFB0A62461046A5F6540129C2EB070D
:1050000067738BA0DB0D570804200945A191B1AE51
:105010000CD92F4A10B2C0561D5A106A881DE86478
:10502000635CF128127383FE90FCD1F7471554AEF0
:1050300042F10B99816B4F0BF538DD494FA5059671
:10504000E69D4EAD1539E172D7467B236DD72BE92E
:10505000A2F944069C7A6DF1A78AC9B85D84E28002
:1050600062BAC014AE4711F1698C398BE1A9BFBC9B
:1050700077D2AC4E5F7E9EA3D4AC23045219D81DC8
:10508000CBCF8607736A617A2478E87BDF1F3141D2
:10509000BC48D0C2E7CB9A5CDD9F0C1DA8677F6738
:1050A000647BCA17C88BE8E77B360D9ACE93F40C65
:1050B00078044A232ABB38A256A7B265B3D24E5F02
:1050C000B49949456DAA02E433F75BFAB804272680
:1050D000BACC36E815E364CB0D2540DBDC9AD62D3F
:1050E00092213B2FC350973ED5D9E7F913EA3CC72D
:1050F000CE9C1EE7112E917BB17FB25220B3C785A3
:10510000035CAD57825C56DD73A289B50148838E7E
:10511000CCC2C62F209F5BB823590B6DD43EB44040
:105120001F994C05AEAE35EB17D585BAF7F58E82D3
:10513000890C0163812B54780735D1BFCB15BDA6EF
:10514000739419293B2BA07C1B4359E7CB7569EB62
:10515000D989F878736E4D9BFACF3BBE8BF5E76229
:10516000C1360AF0C449AF476C0DC457751B97464A
:10517000C441ADC9AB70A134B7A5F91469B8C53144
:10518000004E4F5641E5C337A4EEDD8EEB12B672EA
:105190009ED86AFFF9FA4195F972EBA0C59337D012
:1051A00016D5744D4CE0B04CEBDD012C742FF91783
:1051B00035A7D34EC8BE3CCCCDFBBEBD4574E85C24
:1051C00053E74209E2DFBD08F6F09B191C5A2BF9A0
:1051D000069AB1C837B71B4DCF5A49466321B01064
:1051E000B5815CE196421225B5D0AE159D01DC5E1D
:1051F000D0D39B5A082FF02F903BA2D21FB98DB16C
:105200006906AC8817E982B9D517A96F74BC01BCCF
:1052100024DF4834F129ED334C94B29921B6C5BC52
:105220002B0536BEE8A84F5A2579B5FC1B9B67C2F3
:10523000CEB631E443B6660E83B1C8AB9B22FCB355
:10524000E08BF4F4B9582B10C45F46B9C9BB74396C
:1052500013C2D0433A4B4041872C1F0B6F9CD7633E
:1052600015128514BB89C0515BD2A8E06DDC3A20D1
:10527000AB883A30D600F0544A9595F5B6E5391723
:10528000681250BB90581D69E8AE695B885260FA9D
:10529000B97B33B13C5279CFFCEBB51642DCFEF55D
:1052A0001E91C31BC806A7642D4B6D9517A1767080
:1052B00093232BA1A3FFDFDC1A6EDB4EE52C126ECD
:1052C00009AE636F68541EFECB8F125B68BC57B487
:1052D0008EDDAFF535111D5A2C016B72E899BB0FAD
:1052E00055900ECCDE0E3D7660C6AF572E0BB8D96A
:1052F000D1AE79C2D62B4AF0B83D067AA48790BECB
:10530000FC5DD5C1CB1D9E61656AA89F04DFBDA66B
:105310007706ABE44F3C2CE0EAD6C58812D6577727
:10532000BAC8A0E675D66F50D48FE17F675B565C34
:10533000B2281CEF41264E948E74841DB854557FBC
:10534000855E8A51ABCCD32C0BFB40223E2ECEEA9D
:10535000DD78149A8A9F709270F8882C99561A6F8B
:10536000FF8E493F760376C5B032628FC533937B9B
:10537000E8C6A09EAC73AB9ECD334F9C169641DF22
:10538000541BAABBAE2CC192E2F373F76A1805A9AD
:10539000046C0AA5AB7E64868AFBDA1F1A25B9E87D
:1053A000BE7C346D431BC9DE21C649C3C7F2364FEC
:1053B000ADD1CE1953A4CE832101835181045C3F2A
:1053C00095F1D6FCBEB6B3B7EC06686AE657372A45
:1053D0002B663BC4C8386587A77552C695C1E5964C
:1053E000F70D10D473920B519E15437A23B4229774
:1053F000158DE7A9540D92F4C329EFEC252FBF6555
:10540000A9130A411F09DA66D2222F1302BC80E1D8
:105410005D481B45FA94C2A2F3D4A4857BA4947F73
:10542000F0FFDAEFC92E899CAB1E3BE0912DB5173A
:1054300046B48ACD95BE86069FCD6BAF0EE2321084
:105440006537B7EFF968DC0CCECCF0F024ADCA0DAF
:10545000B1B86EA6A955B81B2F79F16C59E99747D9
:10546000CC3A9F00911EEF17DA230DD8857AA90A4E
:10547000CFB7B0397B4EDD6216DAA757F148BC4290
:1054800008DDF96F47A09FDFC06B2765D6140E605B
:10549000F8987965F9F3F9C1B8B521C0BA61B05A85
:1054A00082E204660C8087534827B088EEA23C391C
:1054B000CE9C6F8181BCA77E8A862C800AB2190996
:1054C0000F72B0EDD65D30F40CABC41AA1BBC0F8BE
:1054D0000A4FB30A7BF2FFA46F00E658D6557F7DD2
:1054E0009CD1F275675BA9EAA90C9E56E2FC66B4F2
:1054F0001D321B9436925D287FC05E11B66BD06D55
:105500009361AC61A26D85B05C94B7AB8891A3A6A2
:10551000F0144BC13ABBA1F258B0EF01BCA379140F
:10552000AAC09B617AF8BF24503003222125A77EB0
:1055300026E9455CBFF42A02EC38DE6B84B1C93A37
:10554000619264A33E10B2082514A8766027F5275F
:1055500044AE06646E7DA710C34954888A40D86360
:10556000812475D19E3A96670D6A12C0F791781121
:10557000D337673B75F08C0C0CBF4899B5241F2EB0
:1055800057762CF04378DAAC41615CDDAA76F6EF11
:10559000696496748B2D95EC782D3B92DE0FDE3B83
:1055A000FD6FB078745DF1C6657C6C018154921218
:1055B000DED75406E0B2D1DC103C997CD10D866474
:1055C000006EB1E632E5D0F22E1E3D5A167664CF5B
:1055D000D6666FDCA1D657969FFCB69B83AA0EB900
:1055E000226C9845476EE30031EEB72C606C601575
:1055F0001B7C358BE112FC2292511B824680600A93
:1056000063694637A7C6F45792368C1E165F1AFF99
:1056100014F81BC447B69DEC0775317F5A7ABD4D0F
:10562000367FDE2779AFFB8E65391E3357FE73CB8D
:105630005D62176A3CF67C2386F18F072A8075032A
:1056400098C199760A9B9EA1F7F2A6752F6DE1CDC0
:105650007A09ACDEADB35DA49C5E3ACFCE56692A22
:1056600072D75353BFECFBA7B866B873A4DB411ADB
:10567000B04F1A2F6EDF89787F5379D0AAB46ECBE2
:10568000EA70B3EBD39B865D32AE3691B045A6107F
:10569000A34F951065FE6E036B7771BD11278012C5
:1056A0009EECEDFEDC3B1C4415D1D92BC2331FBB55
:1056B000A62894404A0843185EA86B785CD03FDE69
:1056C00017875AB7222433FCC05C1CEAEE22353718
:1056D000A724D1E99EEC5DB5BABE5485F504C92274
:1056E000F8111A59265303A01CA20385E68267D736
:1056F0002610C8D3BCD59BB5D3CD602F5759F84DD4
:105700008B6B53197BB094DEA61CE384A83A65DF4B
:105710001D4FD5041D9E61FFD1C57E58A0EDBB4D28
:105720008E103A498334B4E4FD2601908C6C1093BA
:1057300040EA70DE72CED95D7309C10A8FDB26D8CC
:105740001AD973143401BB416F812A52CD1E4D22E8
:10575000CD811661EA737D1FB6672B2D4F9B438762
:105760004C5F074E02217208ADF01B702B1CBFCF9F
:10577000847EC66ED064F579A99D7A24061CD7D4A0
:105780007AA073E961CF119F9BBFA93A38A6D16275
:10579000CD172C2C555C70A1C35AC945C4BB5AD334
:1057A000D95B828EE62AE197B2B589640809D86E82
:1057B0002584AD764C49347E2F8D85C1FEEA901646
:1057C000FC764D4356CA6258F3E1A7DF1D43410DF5
:1057D000D3B6C99A53C31CBF161E7BC9DCB9AB40F4
:1057E000863E1FEBEA3B4A877F532A4CBCF05306A8
:1057F000CEAC4B9B0C2991BC50912098300AE94DBE
:10580000303595A67E8A453B865338F72C6241F0A9
:1058100086928421F8F8D7BEF2053828B1E812350F
:10582000A9BB500D10F8F6D7101FC7FFBDB9E6830E
:105830008BDB0ECD405AC5D2EA54660443F4AFF276
:10584000CB83ADD432FAF20EB7D422EBF479200434
:105850001A6AC06F68E52AC390AF5391187DA67588
:10586000CE3FD5B430721374E57DFD83129E58206F
:105870004A53F371E4740252E5130E9EB4D24853B6
:10588000D686B09DB44988D5465F1FD0FFBD87CC72
:105890001A89F713C021EDA4E5DA44ECDFC631F331
:1058A00026EAFD765BC04CB48868839DD397530E7F
:1058B000609D0F7690FA19F366C8C260CD3D221F35
:1058C00094540FD8F3736AEAE6A5F45367A47828D2
:1058D0009D5FF1C52A114E2F7DC33E400386F327FD
:1058E0002364FF02CD06685EBCFF67473C4C86B26E
:1058F000E635EDAE7B2E27DD3367625F0F8AF93226
:105900009E28DB713948CC65798FD67D303F703366
:105910009B498FBB94DA0B80286ADCC41AE433CF2E
:1059200080E84F81061B58626B8FCCB7405D6D4994
:1059300016AE21E2CB40293C022B1AF7E478A6B739
:105940001FBED08472CFB5E4ABA072D5EF663E4BDC
:105950002F9BAF0BB1A371EA2DC2711708A5C565C6
:10596000131856A0B9A3553BB887CA5D40C839BCC7
:10597000CD6A1B77D5B56916A94E784DD088986247
:105980005AC66F13D0B0F587467A8BFF01074508DA
:1059900084DF631BCECB842A4C916D78B579D12CF2
:1059A0005A4F6ED7AB892BF81BF0B9327F1A647B44
:1059B000DE2E50496801AF1DE88BF05FE20251E234
:1059C000925180AB9A3A0B93E5DA1860809A673669
:1059D000D2A74BFE673D27BD65982491C3BDC7C8BC
:1059E000D6D49E3B59BEC18FDD14642367E341FDCD
:1059F000E47EB7294E99742D690CBE0B068AD70038
:105A0000FDA27572F41678211D197D2CD198032FF3
:105A100085787A97D197C1AD5F600DF7688720F9D7
:105A200097FDFC8569D27BBD14CAE0078238A0CD02
:105A30002429213C724EC02CFA001C7551D90F69E3
:105A400050FEF1B9997E6EF2004FE4CCC1512B3477
:105A5000E92E66461AC02F017C738D83F07B499234
:105A6000EBB79D997868314B236A1A1CBE53580EC8
:105A7000204BA54BF0794EE4162E4DF85DFA71B728
:105A8000829C166CA0608BFC29B95C611C7B8CC568
:105A9000CA717E6B063C63FDD62AFDAB393899E8A6
:105AA00055B9EF21746C866F69137BCD3E823E132E
:105AB000E026CB20B9946460B30DEAD5E0FDAF07D2
:105AC000418E24015B98A354231BF91CCCD6E667B6
:105AD000EFC93338F66A5FFD7259DF8EDED3F28884
:105AE000D1BDCD3BED59FB5CFAF8804574F599A822
:105AF0007E9E1BFCF9667E0DB8159CDDE29D9647E7
:105B0000C28253568A3C169D14428B5EA6215C9637
:105B10001AC4C9D63D763E0187EE549B779C4FD080
:105B200097BAABA22CE1BCDCD9DCC33377F0B18DE2
:105B3000ECCA3D50EF13B2A6D53ABC125300430C49
:105B4000BE368428FA515DC9474B000674E2E5ED84
:105B5000B195DB7205DBC392A5917C9C9DA2EAB650
:105B60002018E4D78134CBDBDF127B3B730A14B1FE
:105B70002E7F9573298B38B327ACF64D2B1C7433CD
:105B80007AFFCE6C99149A0D6B8343FC91C4A828BC
:105B90008C8A23B69F12AAE12CE58082C712FB9F54
:105BA00074BDB2E71706B89BC9D5391A3BFFEB3A6B
:105BB0001D3F00E310ECED7CB79270482CA250C260
:105BC000E3843E47A6883F7D7C3AC21738F2242AF8
:105BD000E97B10B6F3EC9A9CEBC096603CEE10FAB1
:105BE0002B0D89F0FDC051C08EEF1AF4E47EFF97B3
:105BF0001FFB75142472B780AABC891B9E1688A14E
:105C00001FF9FF368827EB6FF8E6B20A53D2226CF1
:105C100077DA7D168E51A9976137641E5C18DE1005
:105C20006B47B3E65B49B05DFC40AA780C463B3558
:105C30003203C7E65EDA4B208898677FD20BEBC051
:105C4000E95FA673135A1466BEB9F5751E67C15B8A
:105C500026C8DC5070438E79FF11F29ABAAAB13887
:105C600034568E53A35554DCCF542354F10CDDEC41
:105C7000385B781F5455D904B6F477D0CF98E9949F
:105C800040D98F8C4F9ECED7C8E2C7D54AB5D72111
:105C900083409A206AB87AC99C41F258890536092E
:105CA0002BD146BDB91F90B3D4DE22F8C45B5FFF91
:105CB000BB84AF43232D6DC69BE2CF85FCDD316CE9
:105CC0006E743D10F99AFB9FBCD350E4D005EBF6FF
:105CD00015679BB36BAD0E0B93712A64C2046F9072
:105CE00017F39DCD381FF4510D5489F9888693AA76
:105CF000B7B0E74F3254684AD7A287A119DBE3C295
:105D00008B4C62B611539F867C230B0B9976A3793B
:105D100030C81010B1F6F93DD1191156EE42940772
:105D2000D9D839E13BA39A5A7AE05E148C74B81C36
:105D300054E9F931C80D9E065C0B9381DB4AF712DA
:105D40005E54CEFFCE65F7990B51D5EA6987BB82C9
:105D50002D4AC6F84A284EA384166A975586E61B34
:105D6000C48534608280E5BA5AA47FF10F32E6C55B
:105D70006F598214254432B2FD914C19F1144E2210
:105D80000ACF09B067172649251EDD67085B9D5BB2
:105D90007ECDBCC8D428F7CEBE276FD7E5B29EB360
:105DA000FD6D15C4762F9BF16FD56451F1AF0B9348
:105DB0006742AAAF695A47A820C23A1913337770CD
:105DC0001039F8ED847615F38DB0C74ACC53CE5315
:105DD000158361D997E252E38DE0D5AD00F6492BEA
:105DE000B44CFE87F4DC3770A5AAD65BBE292488A4
:105DF000596DB49AD43219A0DFD424653EF4D0BED4
:105E00001A3E96074E485392D8D3D08C64D87C9BC8
:105E10007BE5196B986DDD26C38ACF74CBF6F596BA
:105E2000A1D90E832F2A3F341785A4119B4B85746B
:105E3000EF11047ED580D1B1DF359B49DCF2878D2F
:105E4000867936E860F2347C73E95A083C763E077E
:105E5000F1B50C07CE2593E38CEC853405C1E959E7
:105E60009F64A583B391B06B88FD847A17C08D9A27
:105E7000388E558DD4A74FEF4ED3BDA2DE49C885CD
:105E80002B5D91262D0A3BAEF5EB6752DF1B42CE10
:105E9000C57CEACB1C0F6FA5D8B265D78B8652F2B2
:105EA0008DCEB6B731166DDAA828FC219F5F6F3909
:105EB000094B4BA47BADCA4447E183595F3E326E28
:105EC000F12DB1A3434618F169AB38EACB5FD34853
:105ED000D71748C5B4520409FEEBC529244198746C
:105EE000AE92D2C9AD158144686C3E67EE7FC8445E
:105EF0002D7463199E0094B612977BBFC9C499ACE8
:105F00004AAE149B85EA477B09F45D31571DD96A77
:105F1000313A82784DD412018669CE18190876C4B8
:105F2000A68271E4822405B21924737C7D33101695
:105F3000D2CC5D1A8ACE47951C8AD39F99074DEF24
:105F4000314498EA132B72C8A296610B8212980210
:105F5000A11B25E08B1AF1876CF868398C0D0EEBCC
:105F6000D566A99B29CAF29CCDD1CE358F4D0BEFBA
:105F7000ACE0E3AF56A5F419330C4515AF2DED1F7A
:105F80008912616B8BF571AF66FA62CC1EB749B1AD
:105F9000E7B5D8F8D6B747EC7D2169AF2F72195E07
:105FA0005F269ABD2C8541E53CB109F0FB2776C7F9
:105FB000A397A4684340ECA39BD25A91AEB3227935
:105FC000275AAABD371A4F194962D589B355356288
:105FD0003F0859997457E8961601499EC2F30A542E
:105FE0006F4208A446C70F48E819956BC9D5F71842
:105FF000E7B8D24772B294C8F386D7E4DA8D294E57
:00000001FF
